:100000009AC034C2B3C0B2C0B1C0B0C0AFC0AEC0FD
:10001000ADC061C8ABC0AAC0A9C0A8C0A7C0A6C0D7
:10002000A5C0A4C0A3C0B9C7BFC7D5C731C830C811
:10003000E7C72EC82DC82CC82BC82AC829C828C86D
:1000400027C826C8EEC7F1C7F4C7F7C7FAC7FFC766
:1000500003C812C808C810C806C805C804C810C814
:1000600017C816C815C814C813C812C811C810C8B4
:100070000FC80EC80DC80CC80BC80AC809C80BC8E1
:100080000403090412036F00620064006500760037
:100090002E006100740014034100560052002D0030
:1000A00044006F007000650072001203610076006A
:1000B000720064006F007000650072000600FF09A6
:1000C00001A101150026FF0075088501950E0900A4
:1000D000B202018502951E0900B202018503953E18
:1000E0000900B202018504957E0900B2020185056E
:1000F000953E0900B20201C0120101010000000892
:10010000C016DF0500010102000109022200010101
:1001100000806409040000010300000009210101BE
:100120000001223C000705810308000A0853544BD4
:100130003530305F320011241FBECFE5D4E0DEBF82
:10014000CDBF10E0A0E6B0E0E8E5F1E102C0059027
:100150000D92A438B107D9F713E0A4E8B0E001C0CC
:100160001D92A031B107E1F77DD5F4C749CF85B71E
:10017000836085BF8BB780648BBF83EC8093D40290
:100180008093FF028AE58093D3028093FE02089554
:100190001F93CF93DF93DC01162FEA01888184FF40
:1001A00005C0898198E88927898302C08AE5888308
:1001B000AE014E5F5F4FFA01212F8D918193215047
:1001C000E1F7CA01612F4ED11C5F1883DF91CF91F7
:1001D0001F9108954EEF52E0DBDF089543ED52E0AA
:1001E000D7DF08951F93CF93DF936091E4026350AC
:1001F00067FDB9C08091E102CCE0D0E0C81BD10915
:10020000C851DD4F8091E002803118F4CE0129D52C
:10021000A8C08D3209F095C0683009F0A2C083EC07
:100220008093C8028AE580936000109284008881E0
:10023000807621F0CE01F9D4282F70C09A811092D7
:10024000D1028981882321F41092D20222E05FC07A
:10025000853019F49093E50259C0863009F040C00A
:100260008B81813051F1823041F1833021F58A81D7
:10027000882341F480E890E09093E3028093E202C7
:1002800024E02AC0813019F484E890E00EC0823066
:1002900041F486E990E09093E3028093E20224E146
:1002A0001BC08330C1F48AEA90E09093E30280930C
:1002B000E20222E111C0813221F4CE0199D4282F2B
:1002C0000BC0823241F48CEB90E09093E302809378
:1002D000E2022CE301C020E080E4809384001EC091
:1002E000883021F421E087EE92E013C0893019F4C0
:1002F0009093E7020BC08A3011F421E008C08B30E4
:1003000029F483EC8093D4028093FF0220E081EDF6
:1003100092E09093E3028093E20209C02F3F39F408
:10032000888187FD2E8180E88093840006C08F81BC
:10033000882319F48E81821708F0822F8093610040
:1003400010C08091840087FF0CC0CE01C1D48F3FC4
:1003500021F48EE18093600004C0882311F0109294
:1003600061001092E4028091600084FF58C0809187
:1003700061008F3F09F453C0182F893008F018E04E
:10038000811B809361008091C80298E8892780933F
:10039000C802112391F18091840087FF08C089EC85
:1003A00092E0612FCAD4182F893098F526C0209189
:1003B000E2023091E30286FF0DC0A9ECB2E080E0DA
:1003C00090E0F901E80FF91FE491ED9301961817F9
:1003D000C1F708C0912FD901E9ECF2E08D9181932A
:1003E0009150E1F71150812F90E01F5F0196820F2D
:1003F000931F9093E3028093E20289EC92E0612FD5
:1004000031D0612F6C5F6C3041F08FEF80936100D1
:1004100004C08FEF809361006EE16093600094E10F
:1004200080B38C7031F49150D9F71092E50210929C
:10043000DF02DF91CF911F910895A82FB92F80E09F
:1004400090E041E050EA60956F5F58F42D9138EFED
:1004500082279795879510F0842795273F5FC8F3EB
:10046000F3CF0895EADF8D939D930895CF93CFB78F
:10047000CF93C395839BE9F7839B09C0839B07C0F8
:10048000839B05C0839B03C0839B01C0A6C0DF93F1
:10049000C091E102DD27C851DD4F839B02C0DF918F
:1004A000EBCF2F930F931F9300B32FEF03FB20F994
:1004B0004F933F9310B34FEF012703FB21F93BE02C
:1004C00031C04E7F012F10B3216028C0102F4D7F07
:1004D0002260000000B329C04B7F2460012F000080
:1004E00010B32BC010B3477F28602AC04F7E00B3E3
:1004F00020612CC04F7D10B320622FC04F7B00B312
:10050000206432C0422700B349934FEF0000102708
:1005100013FB20F910B31C70C9F1297F91F2012758
:1005200003FB21F900B3237F89F2315058F11027E2
:1005300013FB22F910B3277E79F2012703FB23F97D
:100540002F7C81F200B3102713FB24F92F7971F26D
:1005500000C010B3012703FB25F92F7359F200C027
:1005600000B3102713FB26F9223040F200C010B36D
:10057000012703FB27F9243028F64F77206810B3B2
:100580000000F9CF10E41ABF00271CC03B50319582
:10059000C31BD04010E41ABF0881033C11F10B3497
:1005A00001F12091DF021981110F1213EDCF4A8161
:1005B000441F093659F10D3211F0013E29F74F70F1
:1005C00009F0042F0093E6023F914F911F910F9184
:1005D0002F91DF91CAB7C6FD4CCFCF91CFBFCF913E
:1005E00018952091E602222379F31091E402112359
:1005F000C1F53430C2F13093E4022093E00210914F
:10060000E1023BE0311B3093E1022DC00091E40296
:1006100001303CF50AE54F7049F43091600034FD3B
:1006200024C000936000C8ECD2E023C0433049F0FE
:100630003091D30234FD19C00093D302C4EDD2E04F
:1006400018C03091FE0234FD10C00093FE02CFEFBF
:10065000D2E00FC02795A8F45150A9F4220F000052
:10066000F9CF4AE503C042ED01C0432FC4E1D0E019
:1006700032E011B31C60939A11BB02B320E41CE07A
:100680005F93012756E002BB279520F4515021F4D7
:10069000220FF9CF012756E000003B5A02BBD0F2EF
:1006A000279528F4515029F4220F0000F9CF012793
:1006B00056E0279502BB20F4515021F4220FF9CFC8
:1006C000012756E02991332302BB21F6037F1091C5
:1006D000E502110FC651D04002BB11F01093DF02AA
:1006E00010E41ABF086011B3137F402F437F5F915E
:1006F00000C000C002BB11BB42BB66CF8F988E9872
:1007000097989698C198B898C0988D989598C598DC
:100710000895DF92EF92FF920F931F93CF93DF9391
:10072000EC01E62ED0908500F89402B30F7B10E028
:1007300018C0188188E0F82E17FD006402BB789479
:100740008D2DC2D4F894979A110F0F7BB199116037
:1007500078948D2DB9D4F8949798FA9469F72196E6
:10076000EA94EE2031F77894812FDF91CF911F9199
:100770000F91FF90EF90DF900895AF92BF92CF92CC
:10078000DF92EF92FF920F931F93CF93DF93EC01D1
:100790005B0188811A81811708F4182FCE01039616
:1007A000612FB7DF75010894E11CF11C00E0C12E38
:1007B000DD2412C02C0D3D1D2D5F3F4FCE01820F59
:1007C000931F61E0A6DF982F8981081718F4F701BD
:1007D00091937F01A8950F5F202F30E0888190E0F2
:1007E0008C199D09281739072CF30BC0109286002D
:1007F00086E890E061E08DDFF70181937F01A895A5
:100800000F5F8981081790F3F5011082F7011082BC
:10081000298130E02E5F3F4FC901DF91CF911F91B9
:100820000F91FF90EF90DF90CF90BF90AF90089521
:100830001F93CF93DF93EC01019668816ADF182F35
:100840002881243040F4822F90E0019664E0621BFE
:100850008C0F9D1F5EDF812FDF91CF911F91089537
:1008600064E057DF80E00895AF92BF92CF92DF92AD
:10087000EF92FF920F931F93CF93DF93EC017B01D5
:10088000C42E10928900442389F480910D0387FFC0
:100890000DC08DE4809386001092870080910C0338
:1008A0008093880086E890E064E033DF9881898156
:1008B00057010894A11CB11CF7011082DA80EC01E9
:1008C00000E010E01FC0A89580910B038093870083
:1008D00080910A0380938800CC2041F400FF03C07C
:1008E000F8E0DF2A03C087EFD82201C060D2D0929F
:1008F000860086E890E064E00CDFF50181935F01FB
:100900000F5F1F4F0C171D07F0F2EC0EFD1EF701D5
:1009100011829E012E5F3F4FC901DF91CF911F9140
:100920000F91FF90EF90DF90CF90BF90AF90089520
:100930000F931F938C01FC018081E0DEF80181811F
:10094000B7D31F910F910895DF92EF92FF920F930B
:100950001F93CF93DF93EC0180917A0049818499B2
:1009600002C08DE01CC0882311F0813019F4109270
:10097000850017C0823011F481E011C0833011F47A
:1009800082E00DC090E001969C0135952795359544
:10099000279534E0959587953A95E1F7820F8093F6
:1009A0008500C59A8F9A97988E9A9698C19AB89A08
:1009B000C0988D9A9598842F7BD38091850084D39D
:1009C000C09A8091850080D3C0988A8171D327E036
:1009D000E22EF12CEC0EFD1E10E294E0D92E1DC08B
:1009E000A895C7016E8195DE082F2E81243040F432
:1009F000822F90E007966D2D621B8C0F9D1F89DE64
:100A00008D81081711F480E00DC0979A80918500C0
:100A10005BD397988091850057D3115008F780E0F9
:100A20006DDE80ECDF91CF911F910F91FF90EF90E1
:100A3000DF9008951F937ED310EF06C080910E03C0
:100A4000882311F481E80BC0109386001092870070
:100A500086E890E064E05DDE80FDF0CF80E01F91ED
:100A60000895FF920F931F938C01FC01F080029672
:100A700064E04FDEF8018181882341F0F9E0FF1541
:100A800010F06AE0F62E8F2DD5DF03C08F2D10D326
:100A900080E01F910F91FF9008956F927F928F9247
:100AA0009F92AF92BF92CF92DF92EF92FF920F93FD
:100AB0001F93CF93DF93EC01662EF88019818A8112
:100AC00080FD04C0E4E07E2E08E003C070E2772ED3
:100AD00000E4662099F480910D0387FF0FC08DE438
:100AE000809386001092870080910C038093880089
:100AF0001092890086E890E064E00BDEC12EDF2CC6
:100B000046010894810891085E01EE24FF245CC030
:100B1000A89580910B038093870080910A038093AE
:100B20008800F5018185809389001C81662021F46D
:100B3000177FE0FE02C018603AD11093860086E865
:100B400090E064E0E6DD8A8180FF0CC0E814F904DF
:100B500090F187FF30C08D818093860086E890E019
:100B600064E0D7DD9A81872D8923F1F0F5011185A5
:100B70008F811817F1F088851817D9F08E81877F3B
:100B8000E0FC8860809386008B81D4D206C080917F
:100B90000E03882311F480E80FC086E890E064E03B
:100BA000B8DD8117A1F707C0902319F08B8142DFD0
:100BB00003C08B817DD280E00894A11CB11C8823E6
:100BC00041F40894E11CF11CEC14FD0408F4A0CFDE
:100BD00080E0DF91CF911F910F91FF90EF90DF9018
:100BE000CF90BF90AF909F908F907F906F9008951F
:100BF000FC0180918C00882319F420E030E010C0C3
:100C00008381813021F428EF30E082E109C0823015
:100C100021F02CE131E089E003C02AE031E082E2FA
:100C20003093E3022093E2020895FC0180818076F4
:100C30008032A9F480918C00882389F081818130F1
:100C400011F0893061F4828180938A00853011F43B
:100C500083E001C081E080938B008FEF089580E0F6
:100C6000089508952EE088E190E00FB6F894A895D5
:100C700081BD0FBE21BD81E080938C0018BA80E257
:100C800087BB15BA14BA80E182BB11BA8B9A20E0F7
:100C900048EB5BE004C0A895CA010197F1F7215029
:100CA000D1F78B9883E083BF81E089BF82E88FBD55
:100CB00029E02EBD81E090E09BBD8ABD25BD82E08C
:100CC00083BD40D254DA7894A8958CDAE9D1FCCF70
:100CD0000F931F93CF93DF93FC01162F90918B00FE
:100CE000992321F1892F8150823000F500E068308E
:100CF00009F001E0913011F0EF0109C0818180938A
:100D00008A00EF012296125082E080938B0080913E
:100D10008A00882361F0888185D080918A00815083
:100D200080938A00115019F02196F1CF01E0802FB5
:100D3000DF91CF911F910F910895FF920F931F9311
:100D4000CF93DF938C01F62E90918B00992339F18C
:100D5000892F8150823018F5913019F0E801162F53
:100D60000FC080918A00E8018993D2D091118FEF52
:100D7000F801818321961F2D125082E080938B0011
:100D800080918A00882361F0CFD097FF03C0109232
:100D90008A0006C08883115019F02196F5CFFF24F0
:100DA0008F2DDF91CF911F910F91FF90089580912A
:100DB0000A0390910B03A0910C03B0910D030196CF
:100DC000A11DB11D80930A0390930B03A0930C0304
:100DD000B0930D0308952BE12093AB0120918E0079
:100DE0002093AC019093AD018093AE012EE020934F
:100DF000AF011092C5021092C40206969093C702EA
:100E00008093C6029C0121503040EBEAF1E090E073
:100E100004C0819198272150304021153105C9F730
:100E200090830895282F80910F03882321F4109236
:100E3000A7011092A6018091A6019091A7010097A9
:100E400061F42B3109F060C020938D0081E090E0C7
:100E50009093A7018093A60157C031E08931930791
:100E600008F04EC0FC01E357FF4F2083FC01319690
:100E7000F093A701E093A601E430F105A9F4809175
:100E800090008093A80180918F008093A9018091A8
:100E9000A8019091A90106969093A9018093A801B9
:100EA0008A51914088F12CC0E530F10519F42E30BB
:100EB00039F52AC0E530F10538F18091A80190910B
:100EC000A901E817F90701F590E0ADE8B0E003C02B
:100ED0008D91982731973097D9F71092A7011092EA
:100EE000A601992321F481E08093AA010DC080EB33
:100EF0008093B0018093B10182E090E06CDF04C088
:100F00001092A7011092A60188EC80930F03089518
:100F10002091C6023091C7028091C4029091C5020F
:100F2000281B390BC90108952091C6023091C702D0
:100F30002115310519F4EFEFFFEF19C08091C402BC
:100F40009091C502FC01E555FE4FE081019690931A
:100F5000C5028093C4028217930740F01092C70223
:100F60001092C6021092C5021092C402F0E0CF01A6
:100F70000895CF93DF93C2E0D0E0809192008093F8
:100F8000B0011092B10190E0FC013197ED32F10512
:100F900008F07EC0ED5EFF4F099482EB91E06CE2B9
:100FA00071E0D1D0CBE077C0E09193002091940024
:100FB000E63939F485B5922F9770887F982B95BDC7
:100FC00003C0E73909F423BDF0E0EF71F070EE598A
:100FD000FF4F208360C0E0919300E63919F4E5B536
:100FE000E7700AC0E73911F4E3B506C0F0E0EF712D
:100FF000F070EE59FF4FE081E093B201C3E04BC0C7
:101000008091930080930D038091940080930C0352
:101010008091950080930B038091960080930A0342
:101020003AC083E990E090DC34C083E990E080DC52
:1010300032C083E990E015DD2CC083E990E060E0E8
:1010400009C083E990E061EB71E040E00AC083E908
:1010500090E061E022DD1DC083E990E061EB71E08A
:1010600041E002DC12C083E990E0E2DB8093B20150
:101070001092B301C4E00FC083E990E0F1DB09C036
:1010800083E990E061EB71E078DBEC01219603C02D
:1010900080EC8093B101CE019EDEDF91CF91089567
:1010A0008091AA01882319F01092AA0162DF0895A5
:1010B000982F969596958F5F891B80930E0380914C
:1010C0000E038823E1F70895F89481E080BF82B78A
:1010D000789482B7089578941F920F920FB60F926A
:1010E00011248F93F89480910E03882329F0809126
:1010F0000E03815080930E037894F89480918200BF
:10110000815080938200882371F489E48093820067
:10111000789480910F03882339F080910F038150D8
:1011200080930F0301C078948F910F900FBE0F90A2
:101130001F901895982F9F5F86958695981B909382
:101140000E0308950895FB01DC0105900D92002027
:08115000E1F70895F894FFCFC8
:101158005AFF00000000000000000000000000002E
:10116800000001020A00320001800200AA0000000B
:041178000000010072
:00000001FF
